:020000040000FA
:1000000038210020DD020000E5020000E7020000C8
:10001000E9020000EB020000ED0200000000000019
:10002000000000000000000000000000EF020000DF
:10003000F102000000000000F3020000F5020000E1
:100040006D030000F7020000F7020000F702000055
:10005000F7020000F7020000F7020000F7020000BC
:10006000F7020000F7020000F7020000F7020000AC
:10007000F7020000F7020000F7020000F70200009C
:10008000F7020000C5030000F7020000F7020000BD
:10009000F7020000F7020000F7020000F70200007C
:1000A000F7020000F7020000F7020000F70200006C
:1000B000F7020000F702000000000000000000004E
:1000C000F7020000F7020000F7020000F70200004C
:1000D000F7020000F7020000F7020000F70200003C
:1000E000F7020000F7020000F70200000000000025
:1000F00000000000F702000000000000F70200000E
:1001000000000000000000000000000000000000EF
:1001100000000000000000000000000000000000DF
:1001200000000000000000000000000000000000CF
:1001300000000000000000000000000000000000BF
:1001400000000000000000000000000000000000AF
:10015000000000000000000000000000000000009F
:10016000000000000000000000000000000000008F
:10017000000000000000000000000000000000007F
:10018000000000000000000000000000000000006F
:10019000000000000000000000000000000000005F
:1001A000000000000000000000000000000000004F
:1001B000000000000000000000000000000000003F
:1001C000000000000000000000000000000000002F
:1001D000000000000000000000000000000000001F
:1001E000000000000000000000000000000000000F
:1001F00000000000000000000000000000000000FF
:10020000DFF80CD000F0A0F8004800478D0B00008C
:100210003821002030B450E8012F93B2C489234420
:100220008489A34228BF1B1B0489A34202BFBFF3DA
:100230002F8F002007E0C3EA020340E80134002CBE
:10024000E9D14FF001000A6030BC704750E8012F3F
:10025000C2EA024240E801210029F7D1704730B4D8
:1002600050E8022F1FFAA2F3C488A34202BFBFF3D3
:100270002F8F00200DE0C48923448489A34228BF26
:100280001B1BC2EA034340E80234002CE8D14FF0C4
:1002900001000A6030BC704750E8022FC2EA2242D7
:1002A00040E802210029F7D17047034653E8022FA6
:1002B000D988B2EB324F4FF0000017BF92B241EA3B
:1002C000014142EA014104E05A68B2EB324F08BFF3
:1002D000012043E80212002AE8D17047064880470F
:1002E00006480047FEE7FEE7FEE7FEE7FEE7FEE71B
:1002F000FEE7FEE7FEE7FEE7D5030000010200008F
:1003000040EA01039B0703D009E008C9121F08C097
:10031000042AFAD203E011F8013B00F8013B521E17
:10032000F9D27047D2B201E000F8012B491EFBD28E
:1003300070470022F6E710B513460A4604461946F0
:10034000FFF7F0FF204610BD064C074D06E0E068C1
:1003500040F0010394E8070098471034AC42F6D30C
:10036000FFF752FFFC1000001C11000070B54FF4A5
:100370008076304600F06DFC114CB50560B130461A
:1003800000F06EFC0120C5F80803607920B9012057
:1003900060712168002088474FF48276304600F073
:1003A00058FC00280AD0304600F05AFC0220C5F85C
:1003B00008032168BDE870400120084770BD0000B7
:1003C0000000002002490248091F09680068084728
:1003D0003400002030B54FF0805000228300D0F868
:1003E0003011C3F80C21C3F81021624B1A60624B24
:1003F0001B68624C2360604B1B1D1B68241D23601F
:100400005D4B08331B68241D23605B4B0C331B685A
:10041000241D2360584B10331B68241D2360564B4A
:1004200014331B68241D2360534B18331B68534C33
:1004300020342360504B1C331B68241D23604E4B1B
:1004400020331B68241D23604B4B24331B68241D61
:100450002360494B28331B68241D2360464B2C33F3
:100460001B68241D2360444B30331B68434C4034CD
:100470002360414B34331B68241D23603E4B3833CB
:100480001B68241D23603C4B3C331B68241D2360E8
:10049000394B40331B68241D23600123082902D1F6
:1004A000D0F8344114B1082904D006E0354C344961
:1004B000216005E0D0F8344114B1082904D006E0E9
:1004C000314CFB21216005E0D0F8344114B10829FA
:1004D00008D00EE090F858422C48016864F30301FC
:1004E000016002E0D0F834411CB929494FF4007092
:1004F000086028480168C90702D06FF00101016057
:100500002548016841F470010160BFF34F8FBFF3CC
:100510006F8F4FF01021D1F80002002803DBD1F8D3
:100520000402002822DA1D4C23601D480368002BBA
:10053000FCD01223C1F800320568002DFCD0C1F8B0
:10054000043201680029FCD0226001680029FCD037
:10055000BFF34F8F10487C380168124A01F4E06104
:1005600011430160BFF34F8F00BFFDE70F490E48F5
:10057000086030BD380500400404001020C500406C
:10058000488103008C56004018F50040E40E0040FE
:10059000409602400004004088ED00E004E5014080
:1005A00000E401400400FA050090D0034000002060
:1005B00002E008C8121F08C1002AFAD1704770472C
:1005C000002001E001C1121F002AFBD1704700008A
:1005D00072B609480068C00700D000BEBFF34F8F55
:1005E0000548E4380168054A01F4E06111430160FF
:1005F000BFF34F8F00BFFDE7F0ED00E00400FA0508
:100600000EB500210091CDE901106A4644F20100C7
:10061000FFF7DEFF0EBD0000014800F0D2B8000079
:10062000100000203AB100680129426100D0002189
:1006300001610020704707207047000038B511485D
:1006400008235822416800910F49006800F0C2FA5F
:10065000002815D10D4A69460D4800F0B7F804008E
:100660000ED101210A4800F0FAF80123094A19467F
:10067000074800F07EF80649012008390870204636
:1006800038BD0000DC10000068000020810E000072
:1006900010000020FFFF7F0070B50446007F0D466C
:1006A00008B1002070BDA26100F06CF9401941F161
:1006B0000001C4E90201206900B125612146BDE8BD
:1006C0007040002000F0E4BC00F002B800F008B870
:1006D00072B602480168491C016070472C00002076
:1006E00003490868401E086000D162B670470000E8
:1006F0002C00002070B5084C050009D0103421688A
:10070000002907D008682060496828468847F6E72E
:100710000834F4E770BD000044000020054A0121C0
:1007200020B1012805D19170FFF7E4BF517000207E
:10073000FAE770474400002010B5D0E90234D1E94F
:100740000220D11AA04101D3012010BD002010BD0C
:100750004FF480328A400168C1F848230068C0F82D
:10076000082370474FF4A07202EB810189B200F0B8
:10077000FEB82DE9F04105460E464FF4A07000EB9F
:10078000860081B228684FF48034B440984622F045
:100790007F47C0F808432868C0F84843286800F03D
:1007A000A5FA286800EB8600C0F840752868C0F8F4
:1007B0004443B8F1000F02D02868C0F80443BDE8F4
:1007C000F0810068D0F804057047000010B5437947
:1007D0001B4C44F823204279231D03EBC2021279FB
:1007E0000AB1082010BD02680C88C2F8084590F9CB
:1007F00004208978002A4FEA411106DA02F00F023C
:1008000002F1E02282F8141D03E002F1E02282F8F6
:10081000001490F90410012201F01F0402FA04F4FC
:100820004909890001F1E021C1F80041417903EB58
:10083000C1010A71417943F83100002010BD000068
:100840003000002090F90400012100F01F029140C7
:100850004009800000F1E020C0F8001270470A460D
:10086000022100F07BB84FF4827100F080B800687C
:1008700001210160704700680121416070472DE946
:10088000F05F07460C464FF4A07000EB84001FFA9F
:1008900080FA38684FF48036A6409B4622F07F45A8
:1008A000C0F848633868C0F808633868D0F8048531
:1008B00000EB8402D2F84095C2F840855146386872
:1008C00000F014FAA9EB080020F07F40012806D1BF
:1008D000102000F071FA5146386800F007FA3868C5
:1008E000D0F80485C0F84463A5EB080121F07F41EE
:1008F0003868012900EB840010D0C0F840553868F2
:10090000D0F804156FF07F4C6A1A521E22F07F4215
:10091000ACEB0B03934217D362B118E06D1CC0F827
:100920004055102000F048FA3868D0F804054045DA
:100930000AD10CE000EB84006D1CC0F8405538680B
:10094000D0F80405884202D00D20BDE8F09F0122B6
:100950003146384600F002F80020F6E70368C3F895
:100960004413002A02D00068C0F80413704710B581
:10097000006842581AB100F0B9F9012010BD0020FA
:1009800010BD000010B50B48FFF71BFF094A083ADD
:10099000D2E90434C018D2E9063244F10001C31A86
:1009A00071EB020204D24FF08072801841F1000115
:1009B00010BD0000100000200268134602E08A42C9
:1009C00004D01268002AFAD10B6001607047000061
:1009D0002DE9F04104464078D8B3A178884238D94F
:1009E000E078B0B3E068A0B354211B48FFF7A1FC46
:1009F0001948142221460C30FFF782FC164D0126BF
:100A0000174A6E70A078E1780844A880002028700A
:100A1000E068A860287B85F82000E068A86220696B
:100A20006862FF2085F821000C4805F12001E8628A
:100A300001F11000074600F05BF800280AD1AE7003
:100A4000A078E1780844C1B23846BDE8F04100F032
:100A500047B80720BDE8F081E0000020F810000052
:100A6000650A000070B5194919480A68002A2ADC8D
:100A700002464478D37B928864B1447BE51A954260
:100A800006DC00224270848042690BE0521D0BE0BC
:100A9000D1180CE0847BE518954207D301224270FF
:100AA00084800269002AF1D10A6001E0D11A8180B4
:100AB00001790748303000F013F8002805D0BDE870
:100AC0007040FFF79DBDFF3AEEE770BD3C0000208F
:100AD000E00000200146014800F042B8100100206B
:100AE00082788A4201D207207047C1700020704787
:100AF00070B58261054608788E6828708868A8609D
:100B00008868E860486828624878A870C868002447
:100B1000114A2146E861FFF785FD00281AD111E04E
:100B2000F0070DD02046202C02D24FF0A04102E069
:100B30000A4904F01F0001EB80000322C0F80027DF
:100B40007608641C002EEBD1284600F03DF9012008
:100B50002871002070BD0000F90D00000003005056
:100B600070B50446022020710D462046E16000F079
:100B70002BF9A0682843A06000202075A569A0611A
:100B8000204600F039F90020A56170BD86B000F064
:100B90006FF808B1FFF734FD002000F083F8FFF78D
:100BA0004DFD08B1FFF72CFD142209496846FFF7F7
:100BB000A7FB6846FFF70CFF08B1FFF721FD4FF4D4
:100BC000F030FFF787FF08B1FFF71AFD20BFFDE700
:100BD000C810000010B531B1B2FBF3F403FB1424CC
:100BE0001CB1092010BD0E2010BD01600021416024
:100BF00081608281C381084610BD70B50C460546F0
:100C0000FFF708FB002802D021882868084470BD3F
:100C100010B50A8849888A4203D1FFF73DFB0120BD
:100C200010BD002010BD70B50C460546FFF717FB40
:100C3000002802D061882868084470BD10B50A8871
:100C400049888A4203D1FFF701FB012010BD002033
:100C500010BD00F180400068002800D001207047DE
:100C600008B500F18040002101600068009008BDD7
:100C700070B50A4C207808B185250CE00020A060F2
:100C800060602061E060064800F076F8054600F0FC
:100C90005DF801202070284670BD0000440000204F
:100CA0001D07000070B5104D0446A87838B114B186
:100CB0006168012088470020FFF706FD0CE0002056
:100CC000FFF702FD24B1084821461030FFF774FEFB
:100CD000E86808B900F060F8E868401CE860BDE822
:100CE00070400020FFF7F2BC4400002008B500224D
:100CF00042504058009008BD70B50D460646446805
:100D000004E0B2682946904718B12468206800289A
:100D1000F7D120682860256070BD40680068704782
:100D200041680868002801D002680A6070470246DE
:100D30000020526806E08B4203D108681060012051
:100D400070471A461368002BF5D1704708480068B1
:100D5000012110F0010F06D14FF0E020C02280F8F1
:100D60000024C0F80011034901200860704700000A
:100D700000E100E0180500400649024600200B791A
:100D80000BB1852070470A6001220A7100224A7166
:100D9000704700000000002010B54FF48270FFF78C
:100DA0005FFF02204107C1F80403024901200860E7
:100DB00010BD000008000040002802D00149800159
:100DC00008477047F11000000378026AC16813B148
:100DD000C2F80C1501E0C2F80815002141707047F7
:100DE0000378026AC16813B1C2F8081501E0C2F8BD
:100DF0000C1501214170704770B50446007D052631
:100E000060B12046FFF7E0FF00202075A078E17870
:100E1000411A11FB00F006EB20201FE0A16921B16F
:100E2000204688472079022828D1E578A078A84272
:100E300003D12046FFF7D4FF0EE0204655B1FFF75F
:100E4000CFFFA07810FB05F006EB102020610120F9
:100E5000207504E0FFF7B8FFA078401D20612079DD
:100E600002280BD1E069216922460068FFF714FCD3
:100E7000002803D0BDE87040FFF7C2BB70BD000082
:100E800070B50546FFF7EFFC134C40B1D4E90402FE
:100E90004FF08071411842F10000C4E904100021B4
:100EA0002846FFF75FFC30B1606820B1606800F051
:100EB00087F80020606001212846FFF753FC18B135
:100EC000FFF760FDC4E90601284600F0A5F82846B2
:100ED000BDE8704000F034B80800002070B5054649
:100EE00000200C460870FFF74DFDD5E90223101ACB
:100EF00063EB010300263146361A994112DAB0F548
:100F0000350F03D3FFF788FB0B4942184FF49603C4
:100F100000210A48FFF7B3FC10B10D2806D009E004
:100F2000012070BD00210548FFF712FC284600F0A3
:100F300047F82070002070BDFFFFB40010000020B3
:100F4000F8B51A4C074600261948FFF7E6FED0B15F
:100F5000616871B1D0E902106268D2E90232C91A3F
:100F6000904120D26068007F18B161681048FFF797
:100F7000C3FE00F01FF805466946FFF7AFFF98B1C2
:100F8000606840B10AE0606800280CD13846BDE8CE
:100F9000F840FFF770BC3846FFF769FC65609DF8C4
:100FA00000000028D0D1F8BD6660CDE70800002021
:100FB000E41000000148FFF7B3BE0000E410000099
:100FC00070B50446124800250078F8B1F4B1207FCE
:100FD000E0B1FFF7D7FCD4E90223801A994110D37E
:100FE0002069002600B92677D4E9051088472069D2
:100FF00060B1217F51B1D4E9022110187141C4E9D7
:10100000020121460348FFF777FE0125284670BDFF
:1010100008000020E4100000F8B51B4C6946206869
:10102000FFF701FE00260127184D29E0017821B1C4
:1010300001290CD002291BD114E041680A7FBAB9FA
:101040000F77416810480830FFF756FE10E04168FE
:101050006868814201D16E600AE00B480830FFF7F2
:1010600066FE05E0FFF7A6FF08B10677FAE72F70E6
:1010700069462068FFF7CCFD69462068FFF7D3FD7D
:101080000028D3D1F8BD0000DC10000008000020CB
:10109000F8B50B4C0D46064669462068FFF7ADFDD6
:1010A00058B10670456069462068FFF7C7FD10B16A
:1010B0000448FFF7C7FB0020F8BD0420F8BD00007E
:1010C000DC1000001000002000DC00050000010022
:1010D0000000000000E00100000000505800002067
:1010E0000100060000000000280000203907000071
:1010F0000338FDD870470000C00000201C1100001C
:101100000000002044000000B00500006011000055
:1011100044000020F4200000C00500000000000092
:10112000000000000000000000000000001001406E
:10113000110004000000000000000000000000009A
:10114000000000000000000000000000000000009F
:101150000000000000000000000000000090D0032C
:0400000500000201F4
:00000001FF
